:020000040000FA
:0200000032D0FC
:0200080025D001
:08001800D8CF01F0E8CF00F0A1
:10002000E0CF02F0EACF03F0E9CF04F09EAA02D0BD
:100030009DBAEDD39EA802D09DB8E2D3FF0004C0C4
:10004000E9FF03C0EAFF02C0E0FF00C0E8FF01C013
:10005000D8FF1000EACF05F0E9CF06F0A1A202D048
:10006000A0B22DD0FF00896A8A6A8B6A926A936A6D
:10007000956A966A800E946E070EC16EC26A096A0E
:100080000A6A0B6A0C6A0D6A100E176E080E5EEC97
:1000900005F0080E41EC05F0F40EEE6FEF6F00EE88
:1000A00000F010EE00F0100E176EC9DB03D8CEEC96
:1000B00004F0FDD7010EB16EA282A0821200A192BF
:1000C000200EB26EB36809C089FF0AC08AFF0BC058
:1000D0008BFF0CC08CFF0DC08DFFEE51EF5D14E067
:1000E000EEC0E9FFEA6A030EEE2702E1F40EEE6FBE
:1000F000EF5080EC02F0EE50100FE826E16EE26A5D
:10010000EE50E66EEE50E66E210604E2200602E2B4
:1001100021680992230604E2220602E22368099676
:10012000250604E2240602E22568099A270604E26D
:10013000260602E227680D92290604E2280602E25A
:1001400029680A982B0604E22A0602E22B680A9420
:100150002D0604E22C0602E22D680A902F0604E226
:100160002E0602E22F680C9C310604E2300602E201
:1001700031680C98330604E2320602E233680B98C9
:10018000350604E2340602E235680C94370604E2D0
:10019000360602E237680B92390604E2380602E2BC
:1001A00039680B963B0604E23A0602E23B680C9281
:1001B00006C0E9FF05C0EAFF1100635026E0635066
:1001C00024E00F0EF76E62C0F6FF0800F5501CE049
:1001D000F504086EEA6AEFC0E9FF0850EE6E63505E
:1001E0006324F66E08501724F76E0900F5CF07F068
:1001F0000900F550EE6E0750EE6EE95002E0EF6F29
:100200001200F40EEF6F120012000F0EF76E62C0B4
:10021000F6FF0800F55003E0E806A0D11200120036
:100220007B0E625C01E01200096A0A6A0B6A0C6AC2
:100230000D6A896A8A6A8B6A8C6A8D6A12006250BA
:1002400025EC01F0176E00001200800FE84A700CD8
:10025000E84A600CE84A500CE84A400CE84A300C86
:10026000E84A200C100CF66E0F0EF76E0800F550E1
:1002700012001200030E156EF80E166E120015C055
:10028000EAFF16C0E9FFEE6EEACF15F0E9CF16F0EF
:10029000EA50030807E0EA50040804E0EA500508C1
:1002A00001E0E8D712001550050849E11650000892
:1002B00046E103EEF8F0EE507D0841E1EE507308A0
:1002C0003EE1EE5070083BE1EE50690838E1EE5037
:1002D000720835E1EE50040832E10000EE5025ECE2
:1002E00001F0116E10082BE0EE5033EC01F027E026
:1002F000E8061126800E0E6ED890EE32D8B0EF8E42
:10030000ED52EECF08F0ED50EE6E08C0EEFF040E99
:10031000136E000E106E0E2EEFD7096A0A6A0B6A72
:10032000896A8A6A8B6AA0EC01F0096A0A6A0B6A18
:10033000896A8A6A8B6A020E5EEC05F0120012006E
:10034000000E146E000E126EB6EC01F0400E126E2E
:10035000146EB6EC01F0800E126E146EB6EC01F065
:10036000C00E126E146EB6EC01F012001050F86E52
:100370001150F76E1250F66EA68EA69CA684A68823
:10038000F29E550EA76EAA0EA76EA682F28E0A00E6
:10039000080E0F6E1350EA6E1450E96E080E0E6EC2
:1003A000EE50F56E0F000E2EFBD7A68EA69CA684EF
:1003B000F29E550EA76EAA0EA76EA682F28E0F2E83
:1003C000EDD7A6941050F86E1150F76E1250F66EDD
:1003D0001350EA6E1450E96E400E0E6E0900F5508F
:1003E000EE5E03E10E2EFAD71200100E41EC05F07E
:0203F000FCD738
:10050000060DF950F350F92609840982120009807A
:10051000098612000988098A12000D800D821200D6
:100520000D840A8812000A860A8412000A820A8050
:1005300012000C8E0C8C12000C8A0C8812000B8A94
:100540000B8812000C860C8412000B800B821200A8
:100550000B840B8612000C800C821200186E182679
:1005600018261826F9501850F926099412000990F7
:100570001200099812000D9012000D9412000A96B4
:1005800012000A9212000C9E12000C9A12000B9A92
:1005900012000C9612000B9012000B9412000C909B
:1005A0001200040DF950F350F92609841200098055
:1005B0001200098812000D8012000D8412000A86B4
:1005C00012000A8212000C8E12000C8A12000B8A92
:1005D00012000C8612000B8012000B8412000C809B
:0205E000120007
:10060000040DF950F350F9260982120009961200E0
:10061000099A12000D9212000A9812000A94120010
:100620000A9012000C9C12000C9812000B981200F9
:100630000C9412000B9212000B9612000C921200F6
:1008000066A202D09D981BD482D8AD6E18D4ABB22C
:1008100007D0ABB40AD066B40ED0AE505BD80FD4BC
:10082000AB98AB88FA0E36D80AD4AE50AB98AB88EA
:10083000FC0E30D804D4AE50FB0E2CD800D4C00E21
:1008400094124F0EAF6E240EAC6E900EAB6E666AB5
:10085000616A626A636A606A646A656A09D811D803
:100860009D8A9D889F9A9F98D08EF28CF28E12005E
:10087000000E6A6E6C6E720E6B6E6D6E66906682A6
:100880001200000E6E6E706E820E6F6E716E669448
:10089000668612009D9866B01BD06CC0EAFF6DC0E2
:1008A000E9FFEE6E000EEA6205D0820EE96202D028
:1008B00000EE72F0EACF6CF0E9CF6DF06A506C6236
:1008C00004D06B506D6201D0668066929D881200E4
:1008D0009D88120066B41AD070C0EAFF71C0E9FFAB
:1008E000EE6E000EEA6205D0920EE96202D000EED2
:1008F00082F0EACF70F0E9CF71F06E50706204D0F0
:100900006F50716201D0668466961200120066B262
:100910001CD06AC0EAFF6BC0E9FFEECF69F0000EA1
:10092000EA6205D0820EE96202D000EE72F0EACFF0
:100930006AF0E9CF6BF06C506A6204D06D506B6264
:1009400001D06682669069501200000C9D9A66B6CE
:100950001DD06EC0EAFF6FC0E9FFEECF68F0000E59
:10096000EA6205D0920EE96202D000EE82F0EACF90
:100970006EF0E9CF6FF070506E6204D071506F620C
:1009800001D06686669468509D8A12009D8A000C8C
:1009900066B61200DBDF7EDFFBD7120066B6120000
:1009A000D5DF606E605060AE35D0616E61AC2ED028
:1009B0006150F00BE0082AE06150F00BF00822E1F2
:1009C0006150F20823E06150F1081CE06150F30827
:1009D00019E06150F00844E06150E84A4AD4E84A1E
:1009E00048D4E84A46D4E84A44D4E84A42D4E84ADB
:1009F00040D4E84A3ED4E84A3CD4E84A54D4E84AD1
:100A000038D41200646A010E656E1200646A020E28
:100A1000656E120065BE33D464660FD060C062F0AC
:100A2000642A6450655C01E01200646AD40E615C63
:100A300024E0C40E615C1DE0120060C063F0646AD3
:100A4000940E615C10E0840E615C0FE0B40E615C9A
:100A50000EE0A40E615C0FE0E40E615C10E0120099
:100A6000800E656E07D4DDEF00F005EF01F010EFAA
:100A700001F01FEF01F039EF01F039EF01F039EF2C
:100A800001F0606E616A626A6050636E6150626418
:100A90008A9A62608A8A000000000000000000005C
:100AA00000000000623EF2D7632EF0D7613EECD723
:100AB0008A9A616A626A636A606A1200606E616A39
:100AC000626A6050636E615062648A8A62608A9A68
:100AD0000000000000000000000000000000623E76
:100AE000F2D7632EF0D7613EECD78A8A616A626AD8
:060AF000636A606A120057
:100F000000000000000000000000000000000000E1
:100F100000000000000000000000000000000000D1
:100F200000000000000000000000000000000001C0
:100F300002030405060708090A0B0C0D0E00000049
:100F400000000000000000000000000000000000A1
:100F50000000000000000000000000000000000091
:100F60000000000000000000000000000000000081
:100F70000000000000000000000000000000000071
:1010000000000A000C000F00110014001600190067
:101010001B001E0020002300250028002B002D00AF
:1010200030003200350037003A003C003F004100FC
:101030004400460049004C004E0051005300560049
:1010400058005B005D0060006200650067006A0098
:101050006D006F0072007400770079007C007E00E4
:1010600081008300860088008B008E009000930032
:10107000950098009A009D009F00A200A400A70080
:10108000AA00AC00AF00B100B400B600B900BB00CC
:10109000BE00C000C300C500C800CB00CD00D0001A
:1010A000D200D500D700DA00DC00DF00E100E40068
:1010B000E600E900EC00EE00F100F300F600F800B5
:1010C000FB00FD0000010201050107010A010D01FD
:1010D0000F0112011401170119011C011E01210148
:1010E0002301260128012B012E0130013301350196
:1010F00038013A013D013F014201440147014A01E3
:1011000000000A000C000F00110014001600190066
:101110001B001E0020002300250028002B002D00AE
:1011200030003200350037003A003C003F004100FB
:101130004400460049004C004E0051005300560048
:1011400058005B005D0060006200650067006A0097
:101150006D006F0072007400770079007C007E00E3
:1011600081008300860088008B008E009000930031
:10117000950098009A009D009F00A200A400A7007F
:10118000AA00AC00AF00B100B400B600B900BB00CB
:10119000BE00C000C300C500C800CB00CD00D00019
:1011A000D200D500D700DA00DC00DF00E100E40067
:1011B000E600E900EC00EE00F100F300F600F800B4
:1011C000FB00FD0000010201050107010A010D01FC
:1011D0000F0112011401170119011C011E01210147
:1011E0002301260128012B012E0130013301350195
:1011F00038013A013D013F014201440147014A01E2
:1012000000000A000C000F00110014001600190065
:101210001B001E0020002300250028002B002D00AD
:1012200030003200350037003A003C003F004100FA
:101230004400460049004C004E0051005300560047
:1012400058005B005D0060006200650067006A0096
:101250006D006F0072007400770079007C007E00E2
:1012600081008300860088008B008E009000930030
:10127000950098009A009D009F00A200A400A7007E
:10128000AA00AC00AF00B100B400B600B900BB00CA
:10129000BE00C000C300C500C800CB00CD00D00018
:1012A000D200D500D700DA00DC00DF00E100E40066
:1012B000E600E900EC00EE00F100F300F600F800B3
:1012C000FB00FD0000010201050107010A010D01FB
:1012D0000F0112011401170119011C011E01210146
:1012E0002301260128012B012E0130013301350194
:1012F00038013A013D013F014201440147014A01E1
:1013000000000A000C000F00110014001600190064
:101310001B001E0020002300250028002B002D00AC
:1013200030003200350037003A003C003F004100F9
:101330004400460049004C004E0051005300560046
:1013400058005B005D0060006200650067006A0095
:101350006D006F0072007400770079007C007E00E1
:1013600081008300860088008B008E00900093002F
:10137000950098009A009D009F00A200A400A7007D
:10138000AA00AC00AF00B100B400B600B900BB00C9
:10139000BE00C000C300C500C800CB00CD00D00017
:1013A000D200D500D700DA00DC00DF00E100E40065
:1013B000E600E900EC00EE00F100F300F600F800B2
:1013C000FB00FD0000010201050107010A010D01FA
:1013D0000F0112011401170119011C011E01210145
:1013E0002301260128012B012E0130013301350193
:1013F00038013A013D013F014201440147014A01E0
:1014000000000A000C000F00110014001600190063
:101410001B001E0020002300250028002B002D00AB
:1014200030003200350037003A003C003F004100F8
:101430004400460049004C004E0051005300560045
:1014400058005B005D0060006200650067006A0094
:101450006D006F0072007400770079007C007E00E0
:1014600081008300860088008B008E00900093002E
:10147000950098009A009D009F00A200A400A7007C
:10148000AA00AC00AF00B100B400B600B900BB00C8
:10149000BE00C000C300C500C800CB00CD00D00016
:1014A000D200D500D700DA00DC00DF00E100E40064
:1014B000E600E900EC00EE00F100F300F600F800B1
:1014C000FB00FD0000010201050107010A010D01F9
:1014D0000F0112011401170119011C011E01210144
:1014E0002301260128012B012E0130013301350192
:1014F00038013A013D013F014201440147014A01DF
:1015000000000A000C000F00110014001600190062
:101510001B001E0020002300250028002B002D00AA
:1015200030003200350037003A003C003F004100F7
:101530004400460049004C004E0051005300560044
:1015400058005B005D0060006200650067006A0093
:101550006D006F0072007400770079007C007E00DF
:1015600081008300860088008B008E00900093002D
:10157000950098009A009D009F00A200A400A7007B
:10158000AA00AC00AF00B100B400B600B900BB00C7
:10159000BE00C000C300C500C800CB00CD00D00015
:1015A000D200D500D700DA00DC00DF00E100E40063
:1015B000E600E900EC00EE00F100F300F600F800B0
:1015C000FB00FD0000010201050107010A010D01F8
:1015D0000F0112011401170119011C011E01210143
:1015E0002301260128012B012E0130013301350191
:1015F00038013A013D013F014201440147014A01DE
:1016000000000A000C000F00110014001600190061
:101610001B001E0020002300250028002B002D00A9
:1016200030003200350037003A003C003F004100F6
:101630004400460049004C004E0051005300560043
:1016400058005B005D0060006200650067006A0092
:101650006D006F0072007400770079007C007E00DE
:1016600081008300860088008B008E00900093002C
:10167000950098009A009D009F00A200A400A7007A
:10168000AA00AC00AF00B100B400B600B900BB00C6
:10169000BE00C000C300C500C800CB00CD00D00014
:1016A000D200D500D700DA00DC00DF00E100E40062
:1016B000E600E900EC00EE00F100F300F600F800AF
:1016C000FB00FD0000010201050107010A010D01F7
:1016D0000F0112011401170119011C011E01210142
:1016E0002301260128012B012E0130013301350190
:1016F00038013A013D013F014201440147014A01DD
:1017000000000A000C000F00110014001600190060
:101710001B001E0020002300250028002B002D00A8
:1017200030003200350037003A003C003F004100F5
:101730004400460049004C004E0051005300560042
:1017400058005B005D0060006200650067006A0091
:101750006D006F0072007400770079007C007E00DD
:1017600081008300860088008B008E00900093002B
:10177000950098009A009D009F00A200A400A70079
:10178000AA00AC00AF00B100B400B600B900BB00C5
:10179000BE00C000C300C500C800CB00CD00D00013
:1017A000D200D500D700DA00DC00DF00E100E40061
:1017B000E600E900EC00EE00F100F300F600F800AE
:1017C000FB00FD0000010201050107010A010D01F6
:1017D0000F0112011401170119011C011E01210141
:1017E0002301260128012B012E013001330135018F
:1017F00038013A013D013F014201440147014A01DC
:1018000000000A000C000F0011001400160019005F
:101810001B001E0020002300250028002B002D00A7
:1018200030003200350037003A003C003F004100F4
:101830004400460049004C004E0051005300560041
:1018400058005B005D0060006200650067006A0090
:101850006D006F0072007400770079007C007E00DC
:1018600081008300860088008B008E00900093002A
:10187000950098009A009D009F00A200A400A70078
:10188000AA00AC00AF00B100B400B600B900BB00C4
:10189000BE00C000C300C500C800CB00CD00D00012
:1018A000D200D500D700DA00DC00DF00E100E40060
:1018B000E600E900EC00EE00F100F300F600F800AD
:1018C000FB00FD0000010201050107010A010D01F5
:1018D0000F0112011401170119011C011E01210140
:1018E0002301260128012B012E013001330135018E
:1018F00038013A013D013F014201440147014A01DB
:1019000000000A000C000F0011001400160019005E
:101910001B001E0020002300250028002B002D00A6
:1019200030003200350037003A003C003F004100F3
:101930004400460049004C004E0051005300560040
:1019400058005B005D0060006200650067006A008F
:101950006D006F0072007400770079007C007E00DB
:1019600081008300860088008B008E009000930029
:10197000950098009A009D009F00A200A400A70077
:10198000AA00AC00AF00B100B400B600B900BB00C3
:10199000BE00C000C300C500C800CB00CD00D00011
:1019A000D200D500D700DA00DC00DF00E100E4005F
:1019B000E600E900EC00EE00F100F300F600F800AC
:1019C000FB00FD0000010201050107010A010D01F4
:1019D0000F0112011401170119011C011E0121013F
:1019E0002301260128012B012E013001330135018D
:1019F00038013A013D013F014201440147014A01DA
:101A000000000A000C000F0011001400160019005D
:101A10001B001E0020002300250028002B002D00A5
:101A200030003200350037003A003C003F004100F2
:101A30004400460049004C004E005100530056003F
:101A400058005B005D0060006200650067006A008E
:101A50006D006F0072007400770079007C007E00DA
:101A600081008300860088008B008E009000930028
:101A7000950098009A009D009F00A200A400A70076
:101A8000AA00AC00AF00B100B400B600B900BB00C2
:101A9000BE00C000C300C500C800CB00CD00D00010
:101AA000D200D500D700DA00DC00DF00E100E4005E
:101AB000E600E900EC00EE00F100F300F600F800AB
:101AC000FB00FD0000010201050107010A010D01F3
:101AD0000F0112011401170119011C011E0121013E
:101AE0002301260128012B012E013001330135018C
:101AF00038013A013D013F014201440147014A01D9
:101B000000000A000C000F0011001400160019005C
:101B10001B001E0020002300250028002B002D00A4
:101B200030003200350037003A003C003F004100F1
:101B30004400460049004C004E005100530056003E
:101B400058005B005D0060006200650067006A008D
:101B50006D006F0072007400770079007C007E00D9
:101B600081008300860088008B008E009000930027
:101B7000950098009A009D009F00A200A400A70075
:101B8000AA00AC00AF00B100B400B600B900BB00C1
:101B9000BE00C000C300C500C800CB00CD00D0000F
:101BA000D200D500D700DA00DC00DF00E100E4005D
:101BB000E600E900EC00EE00F100F300F600F800AA
:101BC000FB00FD0000010201050107010A010D01F2
:101BD0000F0112011401170119011C011E0121013D
:101BE0002301260128012B012E013001330135018B
:101BF00038013A013D013F014201440147014A01D8
:101C000000000A000C000F0011001400160019005B
:101C10001B001E0020002300250028002B002D00A3
:101C200030003200350037003A003C003F004100F0
:101C30004400460049004C004E005100530056003D
:101C400058005B005D0060006200650067006A008C
:101C50006D006F0072007400770079007C007E00D8
:101C600081008300860088008B008E009000930026
:101C7000950098009A009D009F00A200A400A70074
:101C8000AA00AC00AF00B100B400B600B900BB00C0
:101C9000BE00C000C300C500C800CB00CD00D0000E
:101CA000D200D500D700DA00DC00DF00E100E4005C
:101CB000E600E900EC00EE00F100F300F600F800A9
:101CC000FB00FD0000010201050107010A010D01F1
:101CD0000F0112011401170119011C011E0121013C
:101CE0002301260128012B012E013001330135018A
:101CF00038013A013D013F014201440147014A01D7
:101D000000000A000C000F0011001400160019005A
:101D10001B001E0020002300250028002B002D00A2
:101D200030003200350037003A003C003F004100EF
:101D30004400460049004C004E005100530056003C
:101D400058005B005D0060006200650067006A008B
:101D50006D006F0072007400770079007C007E00D7
:101D600081008300860088008B008E009000930025
:101D7000950098009A009D009F00A200A400A70073
:101D8000AA00AC00AF00B100B400B600B900BB00BF
:101D9000BE00C000C300C500C800CB00CD00D0000D
:101DA000D200D500D700DA00DC00DF00E100E4005B
:101DB000E600E900EC00EE00F100F300F600F800A8
:101DC000FB00FD0000010201050107010A010D01F0
:101DD0000F0112011401170119011C011E0121013B
:101DE0002301260128012B012E0130013301350189
:101DF00038013A013D013F014201440147014A01D6
:1020000001000100010001000100010001000100C8
:1020100001000100010001000100010001000100B8
:1020200001000100010001000100010001000100A8
:102030000100010001000100010001000100010098
:020000040030CA
:03000100061300E3
:020005008181F7
:060008000FC00FE00F40E5
:00000001FF
